:020000040000FA
:0408000039EF07F0D5
:1008100003B210EF05F0F2B42BEF05F09EB033EF0A
:1008200005F09EB23BEF05F0F2A81AEF04F0F2B229
:1008300025EF04F0F2A620EF04F0F2B022EF04F06E
:1008400017EF07F0F296F290FF00CD90F2929EA083
:100850002FEF04F00101463F2FEF04F0472BA1C119
:10086000A5F1A2C1A6F1A3C1A7F1A4C1A8F19DC1A0
:10087000A1F19EC1A2F19FC1A3F1A0C1A4F199C1B0
:100880009DF19AC19EF19BC19FF19CC1A0F195C1C0
:1008900099F196C19AF197C19BF198C19CF191C1D0
:1008A00095F192C196F193C197F194C198F18DC1E0
:1008B00091F18EC192F18FC193F190C194F189C1F0
:1008C0008DF18AC18EF18BC18FF18CC190F1CECFA9
:1008D00089F1CFCF8AF146C18BF147C18CF1CF6A44
:1008E000CE6A0101466B476B9E90CD800EBC0E8E8A
:1008F0000EBA7EEF04F00E8A17EF07F00E8C0EBED4
:10090000BAEF04F089C18DF18AC18EF18BC18FF1EC
:100910008CC190F18DC191F18EC192F18FC193F193
:1009200090C194F191C195F192C196F193C197F163
:1009300094C198F195C199F196C19AF197C19BF133
:1009400098C19CF199C19DF19AC19EF19BC19FF103
:100950009CC1A0F19DC1A1F19EC1A2F19FC1A3F1D3
:10096000A0C1A4F1A1C1A5F1A2C1A6F1A3C1A7F1A3
:10097000A4C1A8F10101516B526B536B546B8951A7
:1009800051278A5152238B5153238C5154238D511B
:1009900051278E5152238F515323905154239151FB
:1009A00051279251522393515323945154239551DB
:1009B00051279651522397515323985154239951BB
:1009C00051279A5152239B5153239C5154239D519B
:1009D00051279E5152239F515323A0515423A1517B
:1009E0005127A2515223A3515323A4515423A5515B
:1009F0005127A6515223A7515323A8515423D890CD
:100A00005433533352335133D890543353335233D6
:100A10005133D890543353335233513317EF07F0D7
:100A20000392030103EE00F080517F0BE92604C01E
:100A3000EFFF802B8151805D700BD8A48B8200006A
:100A40008051815D700BD8A48B9281518019D8B4EC
:100A5000079017EF07F0F2940101383F17EF07F006
:100A6000392B17EF07F09E900101463F17EF07F073
:100A7000472B17EF07F09E9204005CA140EF05F0B2
:100A8000077C07AC5BEF05F0C274C2B455EF05F00C
:100A9000C3CFADF5C4CFAEF50501D890AE33AD33BD
:100AA000D890AE33AD335CEF05F0C3CF48F1C4CF7F
:100AB00049F15CEF05F0C28207B4C9EF05F03AC115
:100AC0003EF13BC13FF13CC140F13DC141F151C15B
:100AD00055F152C156F153C157F154C158F189C172
:100AE000A9F18AC1AAF18BC1ABF18CC1ACF18DC166
:100AF000ADF18EC1AEF18FC1AFF190C1B0F191C136
:100B0000B1F192C1B2F193C1B3F194C1B4F195C105
:100B1000B5F196C1B6F197C1B7F198C1B8F199C1D5
:100B2000B9F19AC1BAF19BC1BBF19CC1BCF19DC1A5
:100B3000BDF19EC1BEF19FC1BFF1A0C1C0F1A1C175
:100B4000C1F1A2C1C2F1A3C1C3F1A4C1C4F1A5C145
:100B5000C5F1A6C1C6F1A7C1C7F1A8C1C8F1ADC50D
:100B6000AFF5AEC5B0F5AFC5B1F5B0C5B2F5010191
:100B700048514E2749514F23E86A50230D2EC9EFA3
:100B800005F04FC14AF150C14BF14E6B4F6B506BAA
:100B9000078E0201002F17EF07F03C0E006F0501D2
:100BA0002951000AD8B478EF06F005012951010A4D
:100BB000D8B402EF06F005012951020AD8B443EF78
:100BC00006F005012951030AD8B443EF06F00501E8
:100BD0002951040AD8B443EF06F005012951050A4A
:100BE000D8B443EF06F005012951060AD8B443EF03
:100BF00006F005012951070AD8B443EF06F0296B26
:100C000078EF06F005014D670DEF06F04E670DEF2A
:100C100006F04F670DEF06F0506711EF06F078EF22
:100C200006F051C500F152C501F153C502F154C59A
:100C300003F10101010E046F000E056F000E066F37
:100C4000000E076F9FEC1BF000C151F501C152F57A
:100C500002C153F503C154F5006736EF06F0016792
:100C600036EF06F0026736EF06F0036778EF06F01E
:100C70004DC551F54EC552F54FC553F550C554F508
:100C80000E8878EF06F005012A6749EF06F078EF45
:100C900006F00EBE5EEF06F00FA063EF06F0010156
:100CA0003A675AEF06F03B675AEF06F03C675AEF97
:100CB00006F03D675EEF06F063EF06F007AE63EF08
:100CC00006F075EF06F005012B2F78EF06F03C0ECD
:100CD0002B6F2A2F78EF06F00101000E556FE00E02
:100CE000566FA50E576F010E586F05012A6B0E88BF
:100CF000050105015C6B2DB77FEF06F05C810101FA
:100D00007D678AEF06F07E678AEF06F07F678AEFDD
:100D100006F080678EEF06F0BEEF06F081C100F1AD
:100D200082C101F183C102F184C103F10101010E0D
:100D3000046F000E056F000E066F000E076F9FEC2C
:100D40001BF000C181F101C182F102C183F103C135
:100D500084F10067B3EF06F00167B3EF06F00267B6
:100D6000B3EF06F00367BEEF06F07DC181F17EC1EF
:100D700082F17FC183F180C184F10E80D57ED5BE22
:100D800054D0D6CF3AF1D7CF3BF138C13CF1E86A25
:100D9000E8CF3DF10F80010147A7DBEF06F00E9A87
:100DA0000E9C0E9E0101000E516F600E526F3D0EA3
:100DB000536F080E546F01013ABFEBEF06F03B672B
:100DC000EBEF06F03C67EBEF06F03D67EBEF06F06C
:100DD000F28810EF07F0F298516B526B536B546B23
:100DE000896B8A6B8B6B8C6B8D6B8E6B8F6B906B47
:100DF000916B926B936B946B956B966B976B986BF7
:100E0000996B9A6B9B6B9C6B9D6B9E6B9F6BA06BA6
:100E1000A16BA26BA36BA46BA56BA66BA76BA86B56
:100E2000D76AD66A0101386B396B17EF07F002C039
:100E3000E0FF005001C0D8FF1000A6B21DEF07F080
:100E40000CC0A9FF0BC0A8FFA69EA69CA684F29E7C
:100E5000550EA76EAA0EA76EA682F28EA694A6B213
:100E60002FEF07F01200A96EA69EA69CA680A850A0
:100E70001200076A0E6A0F6A0F010D0EC16E860E10
:100E8000C06E030EC26E0F01280E896E130E926E95
:100E9000080E8A6EF30E936E8B6A900E946EF18E2E
:100EA000F19E0D6A01014E6B4F6B506B4A6B4B6BA1
:100EB000F29A01013A6B3B6B3C6B3D6B3E6B3F6BB7
:100EC000406B416B426B436B446B456B386B396BCA
:100ED000D76AD66A0F01280ED56EF28A9D90B00EA1
:100EE000CD6E0101516B526B536B546B556B566B4E
:100EF000576B586B596B5A6B5B6B5C6B466B476BF4
:100F0000CF6ACE6A0E9A0E9C0E9E9D80760ECA6E99
:100F10009D8202013C0E006FCC6A160E33EC07F086
:100F2000E8CF00F1170E33EC07F0E8CF01F1180E0F
:100F300033EC07F0E8CF02F1190E33EC07F0E8CFFD
:100F400003F1010103AFBFEF07F096EC1CF0160EA2
:100F50000C6E00C10BF01DEC07F0170E0C6E01C1FA
:100F60000BF01DEC07F0180E0C6E02C10BF01DEC1F
:100F700007F0190E0C6E03C10BF01DEC07F000C159
:100F80007DF101C17EF102C17FF103C180F100C199
:100F900081F101C182F102C183F103C184F11A0E12
:100FA00033EC07F0E8CF00F11B0E33EC07F0E8CF8D
:100FB00001F11C0E33EC07F0E8CF02F11D0E33EC0B
:100FC00007F0E8CF03F1010103AF15EF08F096EC4D
:100FD0001CF01A0E0C6E00C10BF01DEC07F01B0E7E
:100FE0000C6E01C10BF01DEC07F01C0E0C6E02C163
:100FF0000BF01DEC07F01D0E0C6E03C10BF01DEC89
:1010000007F01A0E33EC07F0E8CF00F11B0E33ECBB
:1010100007F0E8CF01F11C0E33EC07F0E8CF02F146
:101020001D0E33EC07F0E8CF03F100C185F101C1DB
:1010300086F102C187F103C188F1240EAC6E900ED7
:10104000AB6E240EAC6E080EB86E000EB06E1F0EA6
:10105000AF6E0401806B816B0F01900EAB6E0F01C0
:101060009D8A0301806B816BA26B8B9247EC1FF012
:10107000200E33EC07F0E8CF29F505012951FF0ACE
:10108000D8A44AEF08F0296B200E0C6E29C50BF08E
:101090001DEC07F00501010E2A6F3C0E2B6F250E8B
:1010A00033EC07F0E8CF00F1260E33EC07F0E8CF81
:1010B00001F1270E33EC07F0E8CF02F1280E33ECF4
:1010C00007F0E8CF03F1010103AF81EF08F096ECE0
:1010D0001CF0250E0C6E00C10BF01DEC07F0260E67
:1010E0000C6E01C10BF01DEC07F0270E0C6E02C157
:1010F0000BF01DEC07F0280E0C6E03C10BF01DEC7D
:1011000007F000C14DF501C14EF502C14FF503C115
:1011100050F500C151F501C152F502C153F503C1AB
:1011200054F5290E33EC07F0E8CF55F5050156517B
:10113000555DD8A055C556F505012951020A0EE1A5
:1011400081B8AEEF08F00501562FABEF08F055C59A
:1011500056F5AEEF08F081BA66EF22F0210E33ECBF
:1011600007F0E8CF00F1220E33EC07F0E8CF01F1F1
:10117000230E33EC07F0E8CF02F1240E33EC07F036
:10118000E8CF03F1010103AFF4EF08F096EC1CF097
:10119000210E0C6E00C10BF01DEC07F0220E0C6E40
:1011A00001C10BF01DEC07F0230E0C6E02C10BF019
:1011B0001DEC07F0240E0C6E03C10BF01DEC07F0C4
:1011C000210E33EC07F0E8CF00F1220E33EC07F0EC
:1011D000E8CF01F1230E33EC07F0E8CF02F1240E43
:1011E00033EC07F0E8CF03F100C157F501C158F522
:1011F00002C159F503C15AF5F1EC1EF0B3EC1DF034
:1012000003EC1DF005012951030A12E005012951E3
:10121000040A1DE005012951050A24E005012951B0
:10122000060A32E005012951070A38E057EF09F0B4
:10123000A6C500F101010F0E001701010051000ABF
:1012400036E001010051050A32E054EF09F0A6C56D
:1012500000F101010F0E001701010051000A27E003
:1012600054EF09F00501A651000A21E00501A6513D
:10127000150A1DE00501A651300A19E00501A65125
:10128000450A15E054EF09F00501A651000A0FE0E8
:101290000501A651300A0BE054EF09F00501A651F3
:1012A000000A05E054EF09F081BA66EF22F00790DA
:1012B0000001F28EF28C07B037EF19F00EB018EF84
:1012C00014F00EB80AEF0EF00301805181197F0B64
:1012D000D8B437EF19F013EE00F081517F0BE126FF
:1012E000812BE7CFE8FFE00BD8B437EF19F023EEFE
:1012F00082F0A2511F0BD926E7CFDFFFA22BDF50D0
:10130000780AD8A437EF19F0078081C100F182C1B3
:1013100001F183C102F184C103F10101040E046FE4
:10132000000E056F000E066F000E076F9FEC1BF09E
:1013300000AFA4EF09F00101030E816F000E826F70
:10134000000E836F000E846F03018251720AD8B4BD
:1013500018EF14F08251520AD8B418EF14F08251E9
:10136000750AD8B418EF14F08251630AD8B4F3EFB9
:1013700015F08251690AD8B4D3EF10F082517A0A7D
:10138000D8B4E6EF11F08251490AD8B472EF10F0E8
:101390008251500AD8B490EF0FF08251700AD8B43D
:1013A000D3EF0FF08251540AD8B4FEEF0FF0825100
:1013B000740AD8B444EF10F08251730AD8B448EFDD
:1013C00013F08251530AD8B4ADEF13F082514C0A96
:1013D000D8B400EF0AF028EF16F0040114EE00F084
:1013E00080517F0BE12682C4E7FF802B12000D0E97
:1013F000826FEDEC09F00A0E826FEDEC09F012003D
:1014000003018351300AD8B497EF0CF003018351E4
:10141000310AD8B4E5EF0CF003018351320AD8B495
:1014200035EF0DF003018351330AD8B439EF0DF0D5
:1014300003018351340AD8B447EF0DF003018351FF
:10144000350AD8B40FEF0EF0030183514D0AD8B41A
:1014500010EF0BF0030183516D0AD8B42AEF0BF0A3
:1014600003018351490AD8B40FEF0FF003018351F0
:10147000500AD8B441EF0EF003018351540AD8B496
:10148000BAEF0EF003018351630AD8B44AEF0BF0B0
:1014900003018351430AD8B442EF0CF00301835196
:1014A000730AD8B448EF0BF003018351610AD8B432
:1014B0005DEF0AF0D8A428EF16F004014C0E826FFD
:1014C000EDEC09F00401610E826FEDEC09F0B3EC74
:1014D0001DF004012C0E826FEDEC09F096EC1CF06F
:1014E000A5C500F1010139EC1CF025C182F404010D
:1014F000300E8227EDEC09F026C182F40401300E93
:101500008227EDEC09F027C182F40401300E822716
:10151000EDEC09F004012C0E826FEDEC09F096EC75
:101520001CF0A6C500F1010139EC1CF025C182F4C4
:101530000401300E8227EDEC09F026C182F404018B
:10154000300E8227EDEC09F027C182F40401300E41
:101550008227EDEC09F004012C0E826FEDEC09F00E
:1015600096EC1CF0A7C500F1010139EC1CF025C177
:1015700082F40401300E8227EDEC09F026C182F4DA
:101580000401300E8227EDEC09F027C182F404013A
:10159000300E8227EDEC09F004012C0E826FEDEC89
:1015A00009F096EC1CF0A8C500F1010139EC1CF023
:1015B00025C182F40401300E8227EDEC09F026C12A
:1015C00082F40401300E8227EDEC09F027C182F489
:1015D0000401300E8227EDEC09F004012C0E826F1D
:1015E000EDEC09F096EC1CF0ADC500F1010139EC11
:1015F0001CF025C182F40401300E8227EDEC09F0C5
:1016000026C182F40401300E8227EDEC09F027C1D7
:1016100082F40401300E8227EDEC09F03DEF0EF06C
:10162000D7EC1CF084C327F1E4EC1CF05BEC1CF05D
:10163000200E0C6E00C10BF01DEC07F000C129F567
:1016400005012951000A06E005012951010A02E0BD
:1016500059EC1EF004014C0E826FEDEC09F0040110
:101660004D0E826FEDEC09F004012C0E826FEDEC53
:1016700009F096EC1CF029C500F139EC1CF027C1EB
:1016800082F40401300E8227EDEC09F03DEF0EF0FC
:1016900066EF22F004014C0E826FEDEC09F00401BC
:1016A000630E826FEDEC09F003EC1DF004012C0ECB
:1016B000826FEDEC09F05FEC0BF03DEF0EF096EC75
:1016C0001CF0ABC500F10101003B0F0E001739EC17
:1016D0001CF027C182F40401300E8227EDEC09F0E2
:1016E000ABC500F101010F0E0101001739EC1CF030
:1016F00027C182F40401300E8227EDEC09F00401C9
:101700002D0E826FEDEC09F0AAC500F10101003B3E
:101710000F0E001739EC1CF027C182F40401300EC3
:101720008227EDEC09F0AAC500F101010F0E0101BD
:10173000001739EC1CF027C182F40401300E822717
:10174000EDEC09F004012D0E826FEDEC09F0A9C556
:1017500000F10101003B0F0E001739EC1CF027C10E
:1017600082F40401300E8227EDEC09F0A9C500F1E6
:1017700001010F0E0101001739EC1CF027C182F4A2
:101780000401300E8227EDEC09F00401200E826F77
:10179000EDEC09F0A8C500F10F0E0101001739ECBE
:1017A0001CF027C182F40401300E8227EDEC09F011
:1017B0000401200E826FEDEC09F0A7C500F10101D4
:1017C0000101003B0F0E001739EC1CF027C182F419
:1017D0000401300E8227EDEC09F0A7C500F10101EC
:1017E0000F0E0101001739EC1CF027C182F404012F
:1017F000300E8227EDEC09F004013A0E826FEDEC19
:1018000009F0A6C500F10101003B0F0E001739ECED
:101810001CF027C182F40401300E8227EDEC09F0A0
:10182000A6C500F101010F0E0101001739EC1CF0F3
:1018300027C182F40401300E8227EDEC09F0040187
:101840003A0E826FEDEC09F0A5C500F10101003BF5
:101850000F0E001739EC1CF027C182F40401300E82
:101860008227EDEC09F0A5C500F101010F0E00176C
:1018700039EC1CF027C182F40401300E8227EDEC14
:1018800009F0120084C3E8FF0F0BE83AE8CFABF58C
:1018900085C3E8FF0F0B0501AB1387C3E8FF0F0BF0
:1018A000E83AE8CFAAF588C3E8FF0F0B0501AA13B1
:1018B0008AC3E8FF0F0BE83AE8CFA9F58BC3E8FF2E
:1018C0000F0B0501A9138DC3E8FF0F0BE8CFA8F597
:1018D0008FC3E8FF0F0BE83AE8CFA7F590C3E8FF06
:1018E0000F0B0501A71392C3E8FF0F0BE83AE8CFEF
:1018F000A6F593C3E8FF0F0B0501A61395C3E8FFF8
:101900000F0BE83AE8CFA5F596C3E8FF0F0B0501EA
:10191000A51362EC1DF004014C0E826FEDEC09F092
:101920000401430E826FEDEC09F054EF0BF027EC4D
:1019300022F096EC1CF02DC500F139EC1CF00401EE
:101940004C0E826FEDEC09F00401300E826FEDEC6D
:1019500009F004012C0E826FEDEC09F025C182F430
:101960000401300E8227EDEC09F026C182F4040157
:10197000300E8227EDEC09F027C182F40401300E0D
:101980008227EDEC09F004012C0E826FEDEC09F0DA
:1019900096EC1CF02EC500F139EC1CF025C182F448
:1019A0000401300E8227EDEC09F026C182F4040117
:1019B000300E8227EDEC09F027C182F40401300ECD
:1019C0008227EDEC09F03DEF0EF004014C0E826F22
:1019D000EDEC09F00401310E826FEDEC09F0040129
:1019E0002C0E826FEDEC09F025C500F126C501F142
:1019F00027C502F128C503F10101100E046F000E86
:101A0000056F000E066F000E076FCDEC1BF039EC72
:101A10001CF022C182F40401300E8227EDEC09F0A3
:101A200023C182F40401300E8227EDEC09F024C1B9
:101A300082F40401300E8227EDEC09F025C182F416
:101A40000401300E8227EDEC09F026C182F4040176
:101A5000300E8227EDEC09F027C182F40401300E2C
:101A60008227EDEC09F03DEF0EF091EC1FF028EF2E
:101A700016F004014C0E826FEDEC09F00401330EF8
:101A8000826FEDEC09F0C7EC1FF0EFEF0CF00401F2
:101A90004C0E826FEDEC09F00401340E826FEDEC18
:101AA00009F004012C0E826FEDEC09F0D7EC1CF06C
:101AB00084C31EF185C31FF186C320F187C321F1C2
:101AC00088C322F189C323F18AC324F18BC325F192
:101AD0008CC326F18DC327F101011D6BE4EC1CF0D2
:101AE0005BEC1CF0100E046F000E056F000E066F0D
:101AF000000E076FAEEC1BF000C121F501C122F50D
:101B000002C123F503C124F5DAEC21F02EC5A5F5B9
:101B10002FC5A6F530C5A7F531C5A8F532C5A9F57D
:101B200033C5AAF534C5ABF55FEC0BF004012C0E00
:101B3000826FEDEC09F035C500F136C501F137C50E
:101B400002F138C503F10101000E046F000E056FAC
:101B5000010E066F000E076FCDEC1BF039EC1CF088
:101B60001D67B5EF0DF0BAEF0DF004012D0E826F79
:101B7000EDEC09F024C182F40401300E8227EDEC73
:101B800009F025C182F40401300E8227EDEC09F042
:101B900004012E0E826FEDEC09F026C182F40401DF
:101BA000300E8227EDEC09F027C182F40401300EDB
:101BB0008227EDEC09F004012C0E826FEDEC09F0A8
:101BC00096EC1CF039C500F13AC501F152EC17F062
:101BD00004012C0E826FEDEC09F096EC1CF03BC575
:101BE00000F139EC1CF025C182F40401300E82278B
:101BF000EDEC09F026C182F40401300E8227EDECF1
:101C000009F027C182F40401300E8227EDEC09F0BF
:101C10003DEF0EF00E98C7EC1FF03DEF0EF0040103
:101C20004C0E826FEDEC09F00401350E826FEDEC85
:101C300009F004012C0E826FEDEC09F096EC1CF01B
:101C40000784AFC500F1079439EC1CF025C182F47C
:101C50000401300E8227EDEC09F026C182F4040164
:101C6000300E8227EDEC09F027C182F40401300E1A
:101C70008227EDEC09F03DEF0EF0F7EC09F028EFCC
:101C800016F004014C0E826FEDEC09F00401500EC9
:101C9000826FEDEC09F004012C0E826FEDEC09F07F
:101CA00085C31EF186C31FF187C320F188C321F1CC
:101CB00089C322F18AC323F18BC324F18CC325F19C
:101CC0008DC326F18EC327F10101E4EC1CF05BEC1F
:101CD0001CF003018451530A0DE0030184514D0AA5
:101CE00038E00401780E826FEDEC09F0F7EC09F0B2
:101CF00028EF16F00401530E826FEDEC09F0250E6B
:101D00000C6E00C10BF01DEC07F0260E0C6E01C12D
:101D10000BF01DEC07F0270E0C6E02C10BF01DEC52
:101D200007F0280E0C6E03C10BF01DEC07F000C18C
:101D30004DF501C14EF502C14FF503C150F500C18B
:101D400051F501C152F502C153F503C154F51EEF1F
:101D50000FF004014D0E826FEDEC09F0290E0C6EB0
:101D600000C10BF01DEC07F000C155F500C156F5A0
:101D70001EEF0FF004014C0E826FEDEC09F0040130
:101D8000540E826FEDEC09F004012C0E826FEDEC25
:101D900009F084C31EF185C31FF186C320F187C3F8
:101DA00021F188C322F189C323F18AC324F18BC3B3
:101DB00025F18DC326F18EC327F10101E4EC1CF05F
:101DC0005BEC1CF00101000E046F000E056F010EAC
:101DD000066F000E076FAEEC1BF0210E0C6E00C1FB
:101DE0000BF01DEC07F0220E0C6E01C10BF01DEC88
:101DF00007F0230E0C6E02C10BF01DEC07F0240E51
:101E00000C6E03C10BF01DEC07F000C157F501C1CA
:101E100058F502C159F503C15AF51EEF0FF0040140
:101E20004C0E826FEDEC09F00401490E826FEDEC6F
:101E300009F004012C0E826FEDEC09F0250E33EC55
:101E400007F0E8CF00F1260E33EC07F0E8CF01F100
:101E5000270E33EC07F0E8CF02F1280E33EC07F041
:101E6000E8CF03F139EC1CF065EC1AF00401730EB5
:101E7000826FEDEC09F004012C0E826FEDEC09F09D
:101E800096EC1CF0290E33EC07F0E8CF00F139ECAA
:101E90001CF065EC1AF00401730E826FEDEC09F092
:101EA00004012C0E826FEDEC09F051C500F152C512
:101EB00001F153C502F154C503F139EC1CF065EC96
:101EC0001AF00401730E826FEDEC09F004012C0E80
:101ED000826FEDEC09F096EC1CF056C500F139EC80
:101EE0001CF065EC1AF004016D0E826FEDEC09F048
:101EF00004012C0E826FEDEC09F057C500F158C5B6
:101F000001F159C502F15AC503F143EC16F0040181
:101F10002C0E826FEDEC09F0F7EC09F028EF16F0CB
:101F200083C31EF184C31FF185C320F186C321F151
:101F300087C322F188C323F189C324F18AC325F121
:101F40008BC326F18CC327F10101E4EC1CF05BECA0
:101F50001CF0160E0C6E00C10BF01DEC07F0170EF6
:101F60000C6E01C10BF01DEC07F0180E0C6E02C1D7
:101F70000BF01DEC07F0190E0C6E03C10BF01DECFD
:101F800007F000C17DF101C17EF102C17FF103C103
:101F900080F100C181F101C182F102C183F103C16D
:101FA00084F172EF10F083C31EF184C31FF185C367
:101FB00020F186C321F187C322F188C323F189C3AD
:101FC00024F18AC325F18BC326F18CC327F10101CB
:101FD000E4EC1CF05BEC1CF000C17DF101C17EF172
:101FE00002C17FF103C180F100C181F101C182F121
:101FF00002C183F103C184F172EF10F083C31EF1BB
:1020000084C31FF185C320F186C321F187C322F168
:1020100088C323F189C324F18AC325F18CC326F137
:102020008DC327F10101E4EC1CF05BEC1CF0010115
:10203000000E046F000E056F010E066F000E076F95
:10204000AEEC1BF01A0E0C6E00C10BF01DEC07F08D
:102050001B0E0C6E01C10BF01DEC07F01C0E0C6E7C
:1020600002C10BF01DEC07F01D0E0C6E03C10BF04E
:102070001DEC07F000C185F101C186F102C187F1B5
:1020800003C188F172EF10F083C31EF184C31FF106
:1020900085C320F186C321F187C322F188C323F1D0
:1020A00089C324F18AC325F18CC326F18DC327F19E
:1020B0000101E4EC1CF05BEC1CF00101000E046F6C
:1020C000000E056F010E066F000E076FAEEC1BF0E1
:1020D00000C185F101C186F102C187F103C188F118
:1020E00072EF10F0160E33EC07F0E8CF00F1170E88
:1020F00033EC07F0E8CF01F1180E33EC07F0E8CF2E
:1021000002F1190E33EC07F0E8CF03F139EC1CF0C3
:1021100065EC1AF00401730E826FEDEC09F0040116
:102120002C0E826FEDEC09F07DC100F17EC101F152
:102130007FC102F180C103F139EC1CF065EC1AF0AB
:102140000401730E826FEDEC09F004012C0E826F16
:10215000EDEC09F01A0E33EC07F0E8CF00F11B0E9E
:1021600033EC07F0E8CF01F11C0E33EC07F0E8CFB9
:1021700002F11D0E33EC07F0E8CF03F143EC16F04B
:1021800004012C0E826FEDEC09F085C100F186C1CF
:1021900001F187C102F188C103F143EC16F0F7ECBD
:1021A00009F028EF16F00401690E826FEDEC09F0DA
:1021B00004012C0E826FEDEC09F00101040E006F9A
:1021C000000E016F000E026F000E036F39EC1CF061
:1021D00020C182F40401300E8227EDEC09F021C108
:1021E00082F40401300E8227EDEC09F022C182F462
:1021F0000401300E8227EDEC09F023C182F40401C2
:10220000300E8227EDEC09F024C182F40401300E77
:102210008227EDEC09F025C182F40401300E8227FB
:10222000EDEC09F026C182F40401300E8227EDECBA
:1022300009F027C182F40401300E8227EDEC09F089
:1022400004012C0E826FEDEC09F00101060E006F07
:10225000000E016F000E026F000E036F39EC1CF0D0
:1022600020C182F40401300E8227EDEC09F021C177
:1022700082F40401300E8227EDEC09F022C182F4D1
:102280000401300E8227EDEC09F023C182F4040131
:10229000300E8227EDEC09F024C182F40401300EE7
:1022A0008227EDEC09F025C182F40401300E82276B
:1022B000EDEC09F026C182F40401300E8227EDEC2A
:1022C00009F027C182F40401300E8227EDEC09F0F9
:1022D00004012C0E826FEDEC09F00101160E006F67
:1022E000000E016F000E026F000E036F39EC1CF040
:1022F00020C182F40401300E8227EDEC09F021C1E7
:1023000082F40401300E8227EDEC09F022C182F440
:102310000401300E8227EDEC09F023C182F40401A0
:10232000300E8227EDEC09F024C182F40401300E56
:102330008227EDEC09F025C182F40401300E8227DA
:10234000EDEC09F026C182F40401300E8227EDEC99
:1023500009F027C182F40401300E8227EDEC09F068
:1023600004012C0E826FEDEC09F0200EF86EF76A76
:10237000F66A04010900F5CF82F4EDEC09F00900DA
:10238000F5CF82F4EDEC09F00900F5CF82F4EDEC25
:1023900009F00900F5CF82F4EDEC09F00900F5CF62
:1023A00082F4EDEC09F00900F5CF82F4EDEC09F0D0
:1023B0000900F5CF82F4EDEC09F00900F5CF82F4C5
:1023C000EDEC09F0F7EC09F028EF16F08351630A01
:1023D000D8A428EF16F08451610AD8A428EF16F08B
:1023E00085516C0AD8A428EF16F08651410A42E0C4
:1023F0008651440A1BE08651420AD8B44DEF12F0D0
:102400008651350AD8B4B2EF17F08651360AD8B4DF
:1024100007EF18F08651370AD8B470EF18F08651DC
:10242000380AD8B4CEEF18F028EF16F00798079ABC
:1024300004017A0E826FEDEC09F00401780E826FD0
:10244000EDEC09F00401640E826FEDEC09F081A857
:1024500031EF12F00401550E826FEDEC09F036EF0A
:1024600012F004014C0E826FEDEC09F0F7EC09F06C
:1024700028EF16F00788079A04017A0E826FEDECB8
:1024800009F00401410E826FEDEC09F00401610EC8
:10249000826FEDEC09F027EF12F00798078A04012C
:1024A0007A0E826FEDEC09F00401420E826FEDECC2
:1024B00009F00401610E826FEDEC09F027EF12F0D4
:1024C000010159676BEF12F05A676BEF12F05B670F
:1024D0006BEF12F05C6783EF12F0426777EF12F058
:1024E000436777EF12F0446777EF12F0456783EFA9
:1024F00012F00101000E006F000E016F000E026F5E
:10250000000E036F12000101620E046F010E056FD1
:10251000000E066F000E076F59C100F15AC101F19C
:102520005BC102F15CC103F19FEC1BF003BF07EF3D
:1025300013F00101000E046FA80E056F550E066F13
:10254000020E076F59C100F15AC101F15BC102F1DE
:102550005CC103F159C179F15AC17AF15BC17BF1D8
:102560005CC17CF19FEC1BF003BFC0EF12F00101D6
:10257000000E796FA80E7A6F550E7B6F020E7C6F7E
:102580000E0E33EC07F0E8CF0CF10F0E33EC07F032
:10259000E8CF0DF1100E33EC07F0E8CF0EF1110E7D
:1025A00033EC07F0E8CF0FF1E8EC1AF079C104F151
:1025B0007AC105F17BC106F17CC107F19FEC1BF0EC
:1025C0000782ACEC1AF0E8EC1AF00792ACEC1AF0C7
:1025D00079C100F17AC101F17BC102F17CC103F143
:1025E0000792ACEC1AF0CC0E046FE00E056F870E6C
:1025F000066F050E076F9FEC1BF000C10CF101C1C7
:102600000DF102C10EF103C10FF13FEF13F0010113
:10261000800E006F1A0E016F060E026F000E036F20
:1026200042C104F143C105F144C106F145C107F1BE
:102630009FEC1BF003AF20EF13F096EC1CF01200A0
:102640000E0E33EC07F0E8CF0CF10F0E33EC07F071
:10265000E8CF0DF1100E33EC07F0E8CF0EF1110EBC
:1026600033EC07F0E8CF0FF142C100F143C101F1B3
:1026700044C102F145C103F10782ACEC1AF00CC170
:1026800000F10DC101F10EC102F10FC103F1120001
:102690000401730E826FEDEC09F004012C0E826FC1
:1026A000EDEC09F0078455C159F156C15AF157C1F3
:1026B0005BF158C15CF13EC142F13FC143F140C101
:1026C00044F141C145F14AC14CF14BC14DF1079470
:1026D0006EEC13F0F7EC09F028EF16F059C100F199
:1026E0005AC101F15BC102F15CC103F1010139EC96
:1026F0001CF065EC1AF00401630E826FEDEC09F03A
:1027000004012C0E826FEDEC09F042C100F143C1CF
:1027100001F144C102F145C103F1010139EC1CF0A2
:1027200065EC1AF00401660E826FEDEC09F004010D
:102730002C0E826FEDEC09F096EC1CF04CC100F110
:102740004DC101F1010139EC1CF065EC1AF00401F6
:10275000740E826FEDEC09F012000F820401530E2B
:10276000826FEDEC09F004012C0E826FEDEC09F0A4
:1027700083C31EF184C31FF185C320F186C321F1F9
:1027800087C322F188C323F189C324F18AC325F1C9
:102790008BC326F18CC327F10101E4EC1CF05BEC48
:1027A0001CF000C159F101C15AF102C15BF103C132
:1027B0005CF18EC31EF18FC31FF190C320F191C352
:1027C00021F192C322F193C323F194C324F195C361
:1027D00025F196C326F197C327F10101E4EC1CF023
:1027E0005BEC1CF000C142F101C143F102C144F1B4
:1027F00003C145F1D7EC1CF099C323F19AC324F12E
:102800009BC325F19CC326F19DC327F10101E4EC94
:102810001CF05BEC1CF000C14CF101C14DF16EEC01
:1028200013F004012C0E826FEDEC09F01FEF14F091
:102830008251520A03E10E821FEF14F00E92825170
:10284000750A03E10F8426EF14F00F948251550AA4
:1028500003E10F862DEF14F00F9607840FB28AEF75
:1028600014F00FA476EF14F0A9C159F1AAC15AF1DE
:10287000ABC15BF1ACC15CF1ADC15DF1AEC15EF16C
:10288000AFC15FF1B0C160F1B1C161F1B2C162F13C
:10289000B3C163F1B4C164F1B5C165F1B6C166F10C
:1028A000B7C167F1B8C168F1B9C169F1BAC16AF1DC
:1028B000BBC16BF1BCC16CF1BDC16DF1BEC16EF1AC
:1028C000BFC16FF1C0C170F1C1C171F1C2C172F17C
:1028D000C3C173F1C4C174F1C5C175F1C6C176F14C
:1028E000C7C177F1C8C178F17EEF14F055C159F135
:1028F00056C15AF157C15BF158C15CF13EC142F17A
:102900003FC143F140C144F141C145F14AC14CF1DD
:102910004BC14DF107940EA0ACEF14F00101856797
:1029200099EF14F0866799EF14F0876799EF14F028
:1029300088679DEF14F0ACEF14F060EC12F085C1E5
:1029400004F186C105F187C106F188C107F19FEC4A
:102950001BF003BFF0EF15F060EC12F00101000E68
:10296000046F000E056F010E066F000E076FCDECB1
:102970001BF00FA4C3EF14F00401750E826FEDEC91
:1029800009F0C8EF14F00401720E826FEDEC09F04B
:1029900004012C0E826FEDEC09F039EC1CF01D6780
:1029A000D7EF14F00401200E826FDAEF14F0040167
:1029B0002D0E826FEDEC09F024C182F40401300E7B
:1029C0008227EDEC09F025C182F40401300E822744
:1029D000EDEC09F004012E0E826FEDEC09F026C13A
:1029E00082F40401300E8227EDEC09F027C182F455
:1029F0000401300E8227EDEC09F004016D0E826FA8
:102A0000EDEC09F004012C0E826FEDEC09F042C1EF
:102A100000F143C101F144C102F145C103F10101DB
:102A200039EC1CF065EC1AF00401480E826FEDECF5
:102A300009F004017A0E826FEDEC09F004012C0E0E
:102A4000826FEDEC09F059C100F15AC101F15BC18F
:102A500002F15CC103F1010139EC1CF065EC1AF0E4
:102A60000401630E826FEDEC09F004012C0E826FFD
:102A7000EDEC09F059C100F15AC101F15BC102F15D
:102A80005CC103F101010A0E046F000E056F000E18
:102A9000066F000E076FAEEC1BF0000E046F120EF7
:102AA000056F000E066F000E076FCDEC1BF039ECC2
:102AB0001CF01EC182F40401300E8227EDEC09F0F7
:102AC0001FC182F40401300E8227EDEC09F020C111
:102AD00082F40401300E8227EDEC09F021C182F46A
:102AE0000401300E8227EDEC09F022C182F40401CA
:102AF000300E8227EDEC09F023C182F40401300E80
:102B00008227EDEC09F024C182F40401300E822703
:102B1000EDEC09F004012E0E826FEDEC09F025C1F9
:102B200082F40401300E8227EDEC09F026C182F414
:102B30000401300E8227EDEC09F027C182F4040174
:102B4000300E8227EDEC09F00401730E826FEDEC7C
:102B500009F004012C0E826FEDEC09F096EC1CF0EC
:102B60004CC100F14DC101F152EC17F00EB2BCEFB7
:102B700015F00EA0EEEF15F004012C0E826FEDECB7
:102B800009F0200EF86EF76AF66A04010900F5CF25
:102B900082F4EDEC09F00900F5CF82F4EDEC09F0D8
:102BA0000900F5CF82F4EDEC09F00900F5CF82F4CD
:102BB000EDEC09F00900F5CF82F4EDEC09F0090025
:102BC000F5CF82F4EDEC09F00900F5CF82F4EDECDD
:102BD00009F00900F5CF82F4EDEC09F0F7EC09F00B
:102BE0000E9028EF16F00401630E826FEDEC09F0F1
:102BF00004012C0E826FEDEC09F02EEC16F00401AE
:102C00002C0E826FEDEC09F0A1EC16F004012C0EF5
:102C1000826FEDEC09F01DEC17F004012C0E826FB1
:102C2000EDEC09F00101F80E006FCD0E016F660E9C
:102C3000026F030E036F43EC16F004012C0E826F3B
:102C4000EDEC09F033EC17F0F7EC09F028EF16F093
:102C50000301A26B07900F9237EF19F0D8900E0E78
:102C600033EC07F0E8CF00F10F0E33EC07F0E8CFBC
:102C700001F1100E33EC07F0E8CF02F1110E33EC46
:102C800007F0E8CF03F10101000E046F000E056F9D
:102C9000010E066F000E076FCDEC1BF039EC1CF037
:102CA0001EC182F40401300E8227EDEC09F01FC131
:102CB00082F40401300E8227EDEC09F020C182F489
:102CC0000401300E8227EDEC09F021C182F40401E9
:102CD000300E8227EDEC09F022C182F40401300E9F
:102CE0008227EDEC09F023C182F40401300E822723
:102CF000EDEC09F024C182F40401300E8227EDECE2
:102D000009F025C182F40401300E8227EDEC09F0B0
:102D100004012E0E826FEDEC09F026C182F404014D
:102D2000300E8227EDEC09F027C182F40401300E49
:102D30008227EDEC09F004016D0E826FEDEC09F0D5
:102D40001200120E33EC07F0E8CF00F1130E33EC53
:102D500007F0E8CF01F1140E33EC07F0E8CF02F1F1
:102D6000150E33EC07F0E8CF03F101010A0E046FF2
:102D7000000E056F000E066F000E076FAEEC1BF025
:102D8000000E046F120E056F000E066F000E076F27
:102D9000CDEC1BF039EC1CF01EC182F40401300EA6
:102DA0008227EDEC09F01FC182F40401300E822766
:102DB000EDEC09F020C182F40401300E8227EDEC25
:102DC00009F021C182F40401300E8227EDEC09F0F4
:102DD00022C182F40401300E8227EDEC09F023C1F8
:102DE00082F40401300E8227EDEC09F024C182F454
:102DF0000401300E8227EDEC09F004012E0E826FE3
:102E0000EDEC09F025C182F40401300E8227EDECCF
:102E100009F026C182F40401300E8227EDEC09F09E
:102E200027C182F40401300E8227EDEC09F0040181
:102E3000730E826FEDEC09F012000A0E33EC07F00E
:102E4000E8CF00F10B0E33EC07F0E8CF01F10C0EE8
:102E500033EC07F0E8CF02F10D0E33EC07F0E8CFCA
:102E600003F152EF17F0060E33EC07F0E8CF00F154
:102E7000070E33EC07F0E8CF01F1080E33EC07F052
:102E8000E8CF02F1090E33EC07F0E8CF03F152EF7F
:102E900017F0010196EC1CF007844AC100F14BC108
:102EA00001F107940101E80E046F800E056F000E1A
:102EB000066F000E076FAEEC1BF0000E046F040EE1
:102EC000056F000E066F000E076FCDEC1BF0880E2D
:102ED000046F130E056F000E066F000E076F9FEC58
:102EE0001BF00A0E046F000E056F000E066F000E39
:102EF000076FCDEC1BF039EC1CF001011D6786EF6C
:102F000017F00401200E826F89EF17F004012D0ED7
:102F1000826FEDEC09F024C182F40401300E8227A7
:102F2000EDEC09F025C182F40401300E8227EDECAE
:102F300009F026C182F40401300E8227EDEC09F07D
:102F400004012E0E826FEDEC09F027C182F404011A
:102F5000300E8227EDEC09F00401430E826FEDEC98
:102F600009F0120087C31EF188C31FF189C320F145
:102F70008AC321F18BC322F18CC323F18DC324F1C9
:102F80008EC325F190C326F191C327F101011D6B7A
:102F9000E4EC1CF05BEC1CF00101000E046F000E71
:102FA000056F010E066F000E076FAEEC1BF00E0EE4
:102FB0000C6E00C10BF01DEC07F00F0E0C6E01C182
:102FC0000BF01DEC07F0100E0C6E02C10BF01DECA7
:102FD00007F0110E0C6E03C10BF01DEC07F004019D
:102FE0007A0E826FEDEC09F004012C0E826FEDEC8D
:102FF00009F00401350E826FEDEC09F004012C0E8E
:10300000826FEDEC09F02EEC16F036EF12F087C36C
:103010001EF188C31FF189C320F18AC321F18BC33C
:1030200022F18CC323F18DC324F18EC325F190C30B
:1030300026F191C327F101011D6BE4EC1CF05BEC60
:103040001CF0880E046F130E056F000E066F000E45
:10305000076FA3EC1BF0000E046F040E056F000E4B
:10306000066F000E076FAEEC1BF00101E80E046F57
:10307000800E056F000E066F000E076FCDEC1BF083
:103080000A0E0C6E00C10BF01DEC07F00B0E0C6E5F
:1030900001C10BF01DEC07F00C0E0C6E02C10BF021
:1030A0001DEC07F00D0E0C6E03C10BF01DEC07F0CC
:1030B00004017A0E826FEDEC09F004012C0E826F90
:1030C000EDEC09F00401360E826FEDEC09F004011D
:1030D0002C0E826FEDEC09F01DEC17F036EF12F0BC
:1030E00087C31EF188C31FF189C320F18AC321F170
:1030F0008BC322F18CC323F18DC324F18FC325F13F
:1031000090C326F191C327F10101E4EC1CF05BECC4
:103110001CF0000E046F120E056F000E066F000EFD
:10312000076FAEEC1BF001010A0E046F000E056F75
:10313000000E066F000E076FCDEC1BF0120E0C6E2A
:1031400000C10BF01DEC07F0130E0C6E01C10BF06B
:103150001DEC07F0140E0C6E02C10BF01DEC07F015
:10316000150E0C6E03C10BF01DEC07F004017A0E76
:10317000826FEDEC09F004012C0E826FEDEC09F08A
:103180000401370E826FEDEC09F004012C0E826F02
:10319000EDEC09F0A1EC16F036EF12F087C31EF14A
:1031A00088C31FF189C320F18AC321F18BC322F1A7
:1031B0008CC323F18DC324F18EC325F190C326F176
:1031C00091C327F101011D6BE4EC1CF05BEC1CF0DA
:1031D000880E046F130E056F000E066F000E076F4A
:1031E000A3EC1BF0000E046F040E056F000E066FBB
:1031F000000E076FAEEC1BF00101E80E046F800EAD
:10320000056F000E066F000E076FCDEC1BF0060E6B
:103210000C6E00C10BF01DEC07F0070E0C6E01C127
:103220000BF01DEC07F0080E0C6E02C10BF01DEC4C
:1032300007F0090E0C6E03C10BF01DEC07F0040142
:103240007A0E826FEDEC09F004012C0E826FEDEC2A
:1032500009F00401380E826FEDEC09F004012C0E28
:10326000826FEDEC09F033EC17F036EF12F081A825
:10327000F5EF19F007A8AEEF19F00101800E006F0D
:103280001A0E016F060E026F000E036F3EC104F1AD
:103290003FC105F140C106F141C107F19FEC1BF0B0
:1032A00003BFF5EF19F05FEC1AF03EC100F13FC12A
:1032B00001F140C102F141C103F10782ACEC1AF007
:1032C0000CC104F10DC105F10EC106F10FC107F1EA
:1032D000F80E006FCD0E016F660E026F030E036FC6
:1032E0009FEC1BF00E0E0C6E00C10BF01DEC07F0F6
:1032F0000F0E0C6E01C10BF01DEC07F0100E0C6EE2
:1033000002C10BF01DEC07F0110E0C6E03C10BF0A7
:103310001DEC07F00784010196EC1CF04AC100F196
:103320004BC101F107940A0E0C6E00C10BF01DECAD
:1033300007F00B0E0C6E01C10BF01DEC07F00C0E2C
:103340000C6E02C10BF01DEC07F00D0E0C6E03C1EC
:103350000BF01DEC07F00798F5EF19F007AAF5EF51
:1033600019F00784010196EC1CF04AC100F14BC131
:1033700001F10794060E0C6E00C10BF01DEC07F076
:10338000070E0C6E01C10BF01DEC07F0080E0C6E61
:1033900002C10BF01DEC07F0090E0C6E03C10BF01F
:1033A0001DEC07F0078455C100F156C101F157C16A
:1033B00002F158C103F10794120E0C6E00C10BF01C
:1033C0001DEC07F0130E0C6E01C10BF01DEC07F0A5
:1033D000140E0C6E02C10BF01DEC07F0150E0C6EF6
:1033E00003C10BF01DEC07F0079A0401805181190D
:1033F0007F0B0BE09EA809D014EE00F081517F0BEB
:10340000E126E750812B0F01AD6E05012951010A1C
:1034100013E081AA1CEF1AF005012951000A0AE005
:103420000EB81CEF1AF005012A671CEF1AF00EB84F
:103430001CEF1AF066EF22F081B831EF1AF0B3EC0E
:103440001DF005012951020A02E031EF1AF0562F52
:1034500031EF1AF055C556F50501010E2A6F3C0EE5
:103460002B6F5BEF09F00CC100F10DC101F10EC132
:1034700002F10FC103F1000E046F000E056F010E83
:10348000066F000E076FCDEC1BF01DA15EEF1AF06A
:103490001451D8B45EEF1AF00CC100F10DC101F166
:1034A0000EC102F10FC103F1000E046F000E056F93
:1034B0000A0E066F000E076FCDEC1BF01200010123
:1034C0000C6B0D6B0E6B0F6B12001EC182F40401AE
:1034D000300E8227EDEC09F01FC182F40401300E9A
:1034E0008227EDEC09F020C182F40401300E82271E
:1034F000EDEC09F021C182F40401300E8227EDECDD
:1035000009F022C182F40401300E8227EDEC09F0AB
:1035100023C182F40401300E8227EDEC09F024C1AE
:1035200082F40401300E8227EDEC09F025C182F40B
:103530000401300E8227EDEC09F026C182F404016B
:10354000300E8227EDEC09F027C182F40401300E21
:103550008227EDEC09F012000101005305E101534F
:1035600003E1025301E1002B6FEC1BF096EC1CF021
:103570002C51006F2D51016F420E046F4B0E056FE1
:10358000000E066F000E076FAEEC1BF000C104F1D9
:1035900001C105F102C106F103C107F10CC100F13F
:1035A0000DC101F10EC102F10FC103F107B2DDEF50
:1035B0001AF0A3EC1BF0DFEF1AF09FEC1BF000C138
:1035C0000CF101C10DF102C10EF103C10FF11200A6
:1035D00096EC1CF04CC100F14DC101F1060E33EC2C
:1035E00007F0E8CF04F1070E33EC07F0E8CF05F160
:1035F000080E33EC07F0E8CF06F1090E33EC07F0C4
:10360000E8CF07F19FEC1BF000C118F101C119F1DF
:1036100002C11AF103C11BF1290E046F000E056FE0
:10362000000E066F000E076FAEEC1BF0EE0E046F7F
:10363000430E056F000E066F000E076FA3EC1BF024
:1036400018C104F119C105F11AC106F11BC107F136
:10365000AEEC1BF000C110F101C111F102C112F179
:1036600003C113F1120E33EC07F0E8CF04F1130E8F
:1036700033EC07F0E8CF05F1140E33EC07F0E8CF98
:1036800006F1150E33EC07F0E8CF07F10D0E006FD1
:10369000000E016F000E026F000E036FAEEC1BF008
:1036A000180E046F000E056F000E066F000E076FF8
:1036B000CDEC1BF010C104F111C105F112C106F1EE
:1036C00013C107F1A3EC1BF06A0E046F2A0E056FFD
:1036D000000E066F000E076F9FEC1BF01200BF0E6E
:1036E000FA6E200E2D6F2C6BD89000370137023701
:1036F0000337D8B080EF1BF02D2F75EF1BF02C0790
:103700002D070353D8B412000331070B8009326F21
:1037100003390F0B010F2C6F80EC5FF0336F2C051A
:1037200080EC5FF0335D335F2C6B3233D8B02C27E5
:103730002C3332A995EF1BF033512C271200BBEC30
:103740001CF0D8B0120003510719286F7EEC1CF052
:10375000D8900751031928AF800F1200286BA2ECF4
:103760001CF0D8A0B8EC1CF0D8B012008DEC1CF006
:1037700096EC1CF01F0E296FCEEC1CF00B35D8B068
:103780007EEC1CF0D8A00335D8B01200292FBCEF76
:103790001BF028B1A5EC1CF01200286B0451051198
:1037A000061107110008D8A0A2EC1CF0D8A0B8ECB4
:1037B0001CF0D8B01200086B096B0A6B0B6BCEECD7
:1037C0001CF01F0E296FCEEC1CF007510B5DD8A426
:1037D000F6EF1BF006510A5DD8A4F6EF1BF0055179
:1037E000095DD8A4F6EF1BF00451085DD8A009EFDD
:1037F0001CF00451085F0551D8A0053D095F065132
:10380000D8A0063D0A5F0751D8A0073D0B5FD890AE
:103810000081292FE3EF1BF028B1A5EC1CF0286BE9
:10382000A2EC1CF0D890D2EC1CF007510B5DD8A490
:1038300026EF1CF006510A5DD8A426EF1CF00551B6
:10384000095DD8A426EF1CF00451085DD8A035EF1F
:103850001CF0003F35EF1CF0013F35EF1CF0023F3C
:1038600035EF1CF0032BD8B4120028B1A5EC1CF0E6
:1038700012000101286BA2EC1CF0D8B01200D7ECAA
:103880001CF0200E296F003701370237033711EE85
:1038900027F00A0E2A6FE7360A0EE75CD8B0E76E0B
:1038A000E5522A2F4BEF1CF0292F43EF1CF028B1D3
:1038B0001D81D890120001010A0E286F200E296F79
:1038C00011EE1DF028512A6F0A0ED890E652D8B09A
:1038D000E726E7322A2F66EF1CF003330233013369
:1038E0000033292F60EF1CF0E750FF0FD8A00335FD
:1038F000D8B012001DB1A5EC1CF012000451002735
:103900000551D8B0053D01270651D8B0063D022724
:103910000751D8B0073D032712000051086F01512D
:10392000096F02510A6F03510B6F12000101006B06
:10393000016B026B036B12000101046B056B066BDC
:10394000076B12000335D8A012000351800B001F33
:10395000011F021F031F003FB5EF1CF0013FB5EF31
:103960001CF0023FB5EF1CF0032B282B032512009F
:103970000735D8A012000751800B041F051F061F32
:10398000071F043FCBEF1CF0053FCBEF1CF0063FB9
:10399000CBEF1CF0072B282B07251200003701372F
:1039A00002370337083709370A370B37120001018E
:1039B0001D6B1E6B1F6B206B216B226B236B246BAB
:1039C000256B266B276B12001E510F0B1E6F1F51AC
:1039D0000F0B1F6F20510F0B206F21510F0B216F09
:1039E00022510F0B226F23510F0B236F24510F0B0A
:1039F000246F25510F0B256F26510F0B266F275172
:103A00000F0B276F12008984000EC76E220EC66E40
:103A10009E96C69E000EC96EFF0E9EB602D0E82E80
:103A2000FCD79E96C69E000EC96EFF0E9EB602D0B3
:103A3000E82EFCD7C9CFA5F59E96C69E000EC96E8E
:103A4000FF0E9EB602D0E82EFCD7C9CFA6F59E96F3
:103A5000C69E000EC96EFF0E9EB602D0E82EFCD7A1
:103A6000C9CFA7F59E96C69E000EC96EFF0E9EB6E4
:103A700002D0E82EFCD7C9CFA8F59E96C69E000EB0
:103A8000C96EFF0E9EB602D0E82EFCD7C9CFA9F5AD
:103A90009E96C69E000EC96EFF0E9EB602D0E82E00
:103AA000FCD7C9CFAAF59E96C69E000EC96EFF0E22
:103AB0009EB602D0E82EFCD7C9CFABF5899443EC73
:103AC0001FF012008984000EC76E220EC66E9E96ED
:103AD000C69E800EC96EFF0E9EB602D0E82EFCD7A1
:103AE0009E96C69EA5C5C9FFFF0E9EB602D0E82EC3
:103AF000FCD79E96C69EA6C5C9FFFF0E9EB602D0F5
:103B0000E82EFCD79E96C69EA7C5C9FFFF0E9EB69F
:103B100002D0E82EFCD79E96C69EA8C5C9FFFF0E10
:103B20009EB602D0E82EFCD79E96C69EA9C5C9FFB8
:103B3000FF0E9EB602D0E82EFCD79E96C69EAAC562
:103B4000C9FFFF0E9EB602D0E82EFCD79E96C69EF9
:103B5000ABC5C9FFFF0E9EB602D0E82EFCD78994F4
:103B600043EC1FF012008984000EC76E220EC66E51
:103B70009E96C69E070EC96EFF0E9EB602D0E82E18
:103B8000FCD79E96C69E000EC96EFF0E9EB602D052
:103B9000E82EFCD7C9CFA5F59E96C69E000EC96E2D
:103BA000FF0E9EB602D0E82EFCD7C9CFA6F59E9692
:103BB000C69E000EC96EFF0E9EB602D0E82EFCD740
:103BC000C9CFA7F59E96C69E000EC96EFF0E9EB683
:103BD00002D0E82EFCD7C9CFA8F5899443EC1FF09A
:103BE0008984000EC76E220EC66E9E96C69E0F0E6C
:103BF000C96EFF0E9EB602D0E82EFCD79E96C69EDA
:103C0000000EC96EFF0E9EB602D0E82EFCD7C9CFBB
:103C1000ADF5899443EC1FF012008984000EC76E45
:103C2000220EC66E9E96C69E870EC96EFF0E9EB66B
:103C300002D0E82EFCD79E96C69EA5C5C9FFFF0EF2
:103C40009EB602D0E82EFCD79E96C69EA6C5C9FF9A
:103C5000FF0E9EB602D0E82EFCD79E96C69EA7C544
:103C6000C9FFFF0E9EB602D0E82EFCD79E96C69ED8
:103C7000A8C5C9FFFF0E9EB602D0E82EFCD78994D6
:103C800043EC1FF089849E96C69E8F0EC96EFF0E70
:103C90009EB602D0E82EFCD79E96C69EADC5C9FF43
:103CA000FF0E9EB602D0E82EFCD7899443EC1FF09D
:103CB00012008984000EC76E220EC66E9E96C69EA6
:103CC000870EC96EFF0E9EB602D0E82EFCD79E96D8
:103CD000C69E000EC96EFF0E9EB602D0E82EFCD71F
:103CE0009E96C69E800EC96EFF0E9EB602D0E82E2E
:103CF000FCD79E96C69E800EC96EFF0E9EB602D061
:103D0000E82EFCD79E96C69E800EC96EFF0E9EB60C
:103D100002D0E82EFCD7899443EC1FF089849E964C
:103D2000C69E8F0EC96EFF0E9EB602D0E82EFCD73F
:103D30009E96C69E010EC96EFF0E9EB602D0E82E5C
:103D4000FCD7899443EC1FF012008984000EC76EE3
:103D5000220EC66E9E96C69E870EC96EFF0E9EB63A
:103D600002D0E82EFCD79E96C69E000EC96EFF0EAE
:103D70009EB602D0E82EFCD79E96C69E000EC96E57
:103D8000FF0E9EB602D0E82EFCD79E96C69E800EF1
:103D9000C96EFF0E9EB602D0E82EFCD79E96C69E38
:103DA000800EC96EFF0E9EB602D0E82EFCD7899415
:103DB00043EC1FF089849E96C69E8F0EC96EFF0E3F
:103DC0009EB602D0E82EFCD79E96C69E010EC96E06
:103DD000FF0E9EB602D0E82EFCD7899443EC1FF06C
:103DE00012008984000EC76E220EC66E9E96C69E75
:103DF0008F0EC96EFF0E9EB602D0E82EFCD743ECA4
:103E00001FF09E96C69E010EC96EFF0E9EB602D092
:103E1000E82EFCD7899443EC1FF089849E96C69EB9
:103E2000910EC96EFF0E9EB602D0E82EFCD743EC71
:103E30001FF09E96C69EA50EC96EFF0E9EB602D0BE
:103E4000E82EFCD7899443EC1FF012008984000E01
:103E5000C76E220EC66E9E96C69E910EC96EFF0E4E
:103E60009EB602D0E82EFCD743EC1FF09E96C69E6D
:103E7000000EC96EFF0E9EB602D0E82EFCD78994C4
:103E800043EC1FF01200050EE82EFED71200200EA4
:103E9000C66E0501256B266B276B286B899A400E31
:103EA000C76E200EC66E9E96C69E030EC96EFF0E8E
:103EB0009EB602D0E82EFCD79E96C69E27C5C9FFA7
:103EC000FF0E9EB602D0E82EFCD79E96C69E26C553
:103ED000C9FFFF0E9EB602D0E82EFCD79E96C69E66
:103EE00025C5C9FFFF0E9EB602D0E82EFCD79E96D0
:103EF000C69EC952FF0E9EB602D0E82EFCD7898A14
:103F0000C950FF0A02E18EEF1FF0100E2527E86A64
:103F10002623E86A272327A94EEF1FF0220EC66E3C
:103F20001200899A400EC76E200EC66E9E96C69EDF
:103F3000060EC96EFF0E9EB602D0E82EFCD7898A07
:103F4000899A9E96C69EC70EC96EFF0E9EB602D077
:103F5000E82EFCD7898A899A9E96C69E050EC96E60
:103F6000FF0E9EB602D0E82EFCD79E96C69EC95282
:103F7000FF0E9EB602D0E82EFCD7C9B0B5EF1FF0F9
:103F8000898A0501256B266B276B286B12000501BA
:103F9000FE0E2D6F0501000E2D6F03EC1DF0A5C563
:103FA0002EF5A6C52FF5A7C530F5A8C531F5A9C5CD
:103FB00032F5AAC533F5ABC534F5078455C159F1BF
:103FC00056C15AF157C15BF158C15CF13EC142F193
:103FD0003FC143F140C144F141C145F14AC14CF1F7
:103FE0004BC14DF1079460EC12F000C135F501C1F1
:103FF00036F502C137F503C138F50501576708EFFB
:1040000020F0586708EF20F0596708EF20F05A6752
:104010000CEF20F01AEF20F057C504F158C505F158
:1040200059C506F15AC507F101019FEC1BF003BF0A
:1040300088EF20F04CC139F54DC13AF5AFC53BF5DD
:10404000B0C53CF50501100E2C6F899A400EC76E65
:10405000200EC66E9E96C69E060EC96EFF0E9EB6BA
:1040600002D0E82EFCD7898A899A9E96C69E020EB7
:10407000C96EFF0E9EB602D0E82EFCD79E96C69E55
:1040800027C5C9FFFF0E9EB602D0E82EFCD79E962C
:10409000C69E26C5C9FFFF0E9EB602D0E82EFCD7ED
:1040A0009E96C69E25C5C9FFFF0E9EB602D0E82E7D
:1040B000FCD725EE2DF02C2F02D06AEF20F09E9633
:1040C000C69EDECFC9FFFF0E9EB602D0E82EFCD7FB
:1040D0005BEF20F0898A899A9E96C69E050EC96E6E
:1040E000FF0E9EB602D0E82EFCD79E96C69EC95201
:1040F000FF0E9EB602D0E82EFCD7C9B075EF20F0B7
:10410000898A0501100E2527E86A2623E86A2723F5
:10411000120019C502F51AC503F525EE5FF0050179
:104120002C6B16EE00F005010251E1260351D8B0C8
:104130000329E226E7CFE8FF2C0A06E12CC5DEFFC3
:1041400005012C6BACEF20F0E7CFE8FF2A0A0CE06A
:10415000E7CFDEFF05012C2B0501032B023F0307F0
:10416000030E031791EF20F005012D6B2E6B2F6BC3
:10417000306B316B326B336B346B356B366B376B4B
:10418000386B396B3A6B3B6B3C6B3D6B3E6B3F6BFB
:10419000406B416B426B436B446B456B466B476BAB
:1041A000486B496B4A6B4B6B4C6BDDCFE8FF0501ED
:1041B0002C5105E0DDCFE8FF2C2FDAEF20F00501D0
:1041C000DDCF2CF52C5105E0DDCFE8FF2C2FE4EFFF
:1041D00020F00501DDCF2CF52C5105E0DDCFE8FF07
:1041E0002C2FEEEF20F011EE27F00101D7EC1CF0A0
:1041F0000501DDCF2CF52C5105E0DDCFE5FF2C2F9F
:10420000FDEF20F00101E4EC1CF05BEC1CF000C1C0
:104210002EF501C12FF502C130F50501DDCF2CF5DA
:104220002C5105E0DDCFE8FF2C2F12EF21F0050126
:10423000DDCF2CF52C5105E0DDCFE8FF2C2F1CEF56
:1042400021F00501DDCF2CF52C5107E0DDCFE8FF93
:10425000E8A82D852C2F26EF21F011EE27F0010183
:10426000D7EC1CF00501DDCF2CF52C5114E0DDCF8F
:10427000E5FFDDCFE5FFDDCFE5FFDDCFE5FFDDCFFE
:10428000E8FFDDCFE5FFDDCFE5FFDDCFE5FFDDCFEB
:10429000E5FFDDCFE5FF0101E4EC1CF05BEC1CF079
:1042A00000C138F501C139F502C13AF503C13BF54A
:1042B0000501DDCF2CF52C5107E0DDCFE8FFE8A8A4
:1042C0002D832C2F5DEF21F011EE27F00101D7ECAB
:1042D0001CF00501DDCF2CF52C5105E0DDCFE5FF0D
:1042E0002C2F6EEF21F0010122C123F121C122F117
:1042F00020C121F11FC120F1E4EC1CF05BEC1CF0AB
:1043000000C134F501C135F502C136F503C137F5F9
:104310000501DDCF2CF52C5107E0DDCFE8FF2C2F78
:104320008DEF21F0E8B02D8711EE27F00101D7ECD9
:104330001CF0DDCFE8FFDDCFE8FFDDCFE8FFDDCF0C
:10434000E8FFDDCFE8FFDDCFE5FFDDCFE5FFDDCF27
:10435000E5FFDDCFE5FFDDCFE5FFDDCFE5FFE4ECF9
:104360001CF05BEC1CF000C131F501C132F502C15B
:1043700033F5078455C159F156C15AF157C15BF164
:1043800058C15CF13EC142F13FC143F140C144F12B
:1043900041C145F14AC14CF14BC14DF1079460EC6C
:1043A00012F000C13CF501C13DF502C13EF503C16B
:1043B0003FF5120021C500F122C501F123C502F12C
:1043C00024C503F1899A400EC76E200EC66E9E96D4
:1043D000C69E0B0EC96EFF0E9EB602D0E82EFCD70D
:1043E0009E96C69E02C1C9FFFF0E9EB602D0E82E61
:1043F000FCD79E96C69E01C1C9FFFF0E9EB602D095
:10440000E82EFCD79E96C69E00C1C9FFFF0E9EB641
:1044100002D0E82EFCD79E96C69EC952FF0E9EB6CD
:1044200002D0E82EFCD725EE2DF00501100E2C6FE2
:104430009E96C69EC952FF0E9EB602D0E82EFCD7AD
:10444000C9CFDEFF2C2F18EF22F0898A1200899A3B
:10445000400EC76E200EC66E9E96C69E900EC96E0A
:10446000FF0E9EB602D0E82EFCD79E96C69E000E8A
:10447000C96EFF0E9EB602D0E82EFCD79E96C69E51
:10448000000EC96EFF0E9EB602D0E82EFCD79E9697
:10449000C69E000EC96EFF0E9EB602D0E82EFCD757
:1044A0009E96C69EC952FF0E9EB602D0E82EFCD73D
:1044B000C9CF2DF59E96C69EC952FF0E9EB602D05C
:1044C000E82EFCD7C9CF2EF5898A1200B3EC1DF077
:1044D000F29CF29E8B948A86899CC69AC2908A949A
:1044E000898A9482948C720ED36ED3A4FED7899657
:1044F0008A909390FF0EE8CF00F0E82EFED7002EB2
:10450000FCD78150F294F29A9E909D909E929D923B
:0E451000F298F292F290F286F28E0300FF0013
:10BF0000E844F926000C160C2B0C3F0C520C640C68
:10BF1000760C860C960CA50CB30CC10CCF0CDC0C6B
:06BF2000E80CF40C000C1B
:00000001FF
